:100000000C9451090C946E090C946E090C946E09B1
:100010000C946E090C94CE1C0C946E090C946E0911
:100020000C946E090C946E090C946E090C946E0974
:100030000C946E090C946E090C946E090C94792C36
:100040000C946E090C946E090C946E090C946E0954
:100050000C946E090C946E090C946E090C946E0944
:100060000C946E090C946E090C946E090C946E0934
:100070000C946E090C946E090C946E090C946E0924
:100080000C946E090C946E090C946E0948545450EB
:100090002F312E3020323030204F6B0D0A536572D5
:1000A0007665723A2038426974416D4574686572AC
:1000B0006E6574202841544D45474131323829201E
:1000C0006279204343432D41432E64650D0A436FFB
:1000D0006E6E656374696F6E3A20636C6F73650D45
:1000E0000A436F6E74656E742D547970653A206999
:1000F0006D6167652F706E670D0A0D0A89504E4756
:100100000D0A1A0A0000000D494844520000001070
:100110000000001008020000009091683600000105
:10012000F44944415428CF9592CB4A23511086BFBD
:100130003E7D92D3C9E934ADB9C8CC38E3851010FF
:10014000048520B81FE6015CB812B7EE059FC617FC
:10015000F00D1417C6852B17821085080D1294A177
:1001600035D74ED286899D388B441D67355314058B
:1001700005F5513F55BFE1791EFF13F2CFA6D3E934
:10018000542A15CFF39ACDA6943297CB2D2C2CCC94
:10019000CFCF4F4D4DBDCD186F1BAEAEAE4E4E4EB8
:1001A0007ABD9E65594A2929A56DDBF1785C2955F0
:1001B00028149696963E6C2897CB070707A669C623
:1001C000E3712FF26E9F6FA592732F736B99353B7E
:1001D000663F3C3C0063460241101C1E1E02DD517E
:1001E000F7549D86A9100B222A51E5F8EE78E7DB3B
:1001F000CEBABDDEEFF7DBEDB6EBBA02B8BEBEEEAF
:1002000076BB40C929859F43166111E620070EFB86
:10021000F7FBFEC8975206410008E0E6E64629E5EE
:1002200027FC27E7892C7C812CE4C00507121CF9E8
:1002300047AEEB1A86319154ABD5945277CF7758AD
:1002400060810001C66B959CFD3CD35A0B21268032
:10025000699A80699844F00B066040042FEF17D725
:100260005A8F46A389A4999919ADF56C6C9608BA72
:100270005087260410C2108614BF16D3E974369B2B
:100280009D00F97C3E168BADBAABF4A1054DA84399
:1002900003420861C0D6DA562A959252BE034AA993
:1002A0008C95D9CE6CD38316745EB3CFE6F2E6EEAE
:1002B000F75DADF518987CFAF2F2B25AAD0A211E3C
:1002C000792CB54AE7F57360E5D3CAC6F2C6DE8F6E
:1002D0003DAD751445D56AF583352E2E2E822090BE
:1002E000523A8E934C2693C9E4F4F4B46DDB8944FE
:1002F000C2B6ED46A31145D107F3158BC55AADE63D
:10030000FBFE703814428C6F32180CA494636BFCA3
:100310006DBE7F8CDF43E4C2C6455F10BA000000AB
:100320000049454E44AE42608200485454502F313B
:100330002E3020323030204F6B0D0A5365727665B7
:10034000723A2038426974416D45746865726E6511
:1003500074202841544D4547413132382920627973
:10036000204343432D41432E64650D0A436F6E6E57
:10037000656374696F6E3A20636C6F73650D0A4331
:100380006F6E74656E742D547970653A20696D6175
:1003900067652F706E670D0A0D0A89504E470D0A6A
:1003A0001A0A0000000D49484452000000100000E5
:1003B0000010080200000090916836000002124907
:1003C00044415428CF9592CF6A1A5114C6BFDC7BA2
:1003D000C78973471D1562895012349A59347F308A
:1003E0008B24CBD06D1F20E471DA77F1010A598498
:1003F00086EE0381808A09B90C1D5A3A3A63C41B00
:10040000C79951C7A10B256DBA6ACFEEC0F9F8CED6
:10041000F9CE6F4D0881FF29F667F3FCFC7C7F7FE6
:100420002F84180E878CB18D8D8DEDEDEDADADADBA
:100430007C3EFF32B3F6E2D06EB7AFAFAF7DDF5F89
:100440005F5F57559531A6EB7A2A955255B556AB55
:1004500099A6F9CAA1D56A359B4D4A692A95EA1D24
:10046000F6FA477DCE78F167D1FC66EA33BDDFEF5F
:1004700003586A180029E5E5E52580C008AC4FD689
:1004800066617317BB11A2F05D7885ABD32FA7E629
:1004900077330CC3D16864180603D0E974C6E3311E
:1004A00000E7A3735C38AEA39E43CE87EFC0B16074
:1004B000DDBCBF297F2D1B23434AB9123C3C3CA81D
:1004C000AA3A381A948BE53AEAFBD82720010205AC
:1004D000CA1CF30851DB6CEF75F796CB13009EE74F
:1004E000A9AA3A381EE491CF214740080805656063
:1004F000145483D67DD3E59C673299D50D94520070
:100500009CF208910F3F40404123440992973439AF
:10051000E74992AC04A552C9F77DE387111E860E08
:100520001C06A64049900C3088104D3135E766B165
:10053000580430994C08806AB5AA284AE5B1E2C24D
:10054000B56059B0048405CB85EBC2959067CA5954
:100550002693618CAD1CAAD5AA108287FCE0F341DA
:10056000E743678A691A6900534C2564038D739CBD
:1005700083633E9FFFFEF4DDDD9D6DDB8410BFE2F3
:100580008B7D21DE0A003BC1CEC9E2E4825C70CEE5
:10059000E338B66DFB151AB7B7B7524AC658369B43
:1005A000D5344DD3B442A1A0EB7A3A9DD675FDE97E
:1005B000E9298EE357F0351A0DCFF37ABDDE62B12B
:1005C00020842C3399CD668CB1251A7FC3F78FF523
:1005D0000B9C04E839D42369490000000049454ECA
:1005E00044AE42608200485454502F312E302032A5
:1005F0003030204F6B0D0A5365727665723A2038A1
:10060000426974416D45746865726E657420284155
:10061000544D4547413132382920627920434343C4
:100620002D41432E64650D0A436F6E6E65637469D8
:100630006F6E3A20636C6F73650D0A436F6E74655D
:100640006E742D547970653A20746578742F6874CF
:100650006D6C0D0A0D0A3C68746D6C3E0D0A20200D
:100660003C686561643E0D0A202020203C7469745A
:100670006C653E38426974416D45746865726E659B
:10068000743C2F7469746C653E0D0A202020203C58
:100690006D65746120687474702D65717569763D3F
:1006A00022707261676D612220636F6E74656E7473
:1006B0003D226E6F2D6361636865223E0D0A202026
:1006C0003C2F686561643E0D0A20203C626F6479AE
:1006D000206267636F6C6F723D222344434443443E
:1006E000432220746578743D22233030303030301E
:1006F00022206C696E6B3D22233030303043302233
:1007000020616C696E6B3D222330303030433022E3
:1007100020766C696E6B3D222330303030433022BE
:100720003E0D0A202020203C68313E384269744149
:100730006D45746865726E65743C2F68313E0D0AB4
:100740002020202020203C7461626C6520626F7242
:100750006465723D2231222063656C6C7061646453
:10076000696E673D2233223E0D0A20202020202082
:1007700020203C74723E0D0A2020202020202020C2
:1007800020203C746420616C69676E3D2263656E55
:10079000746572223E3C623E706F72743C2F623E02
:1007A0003C2F74643E0D0A20202020202020202091
:1007B000203C746420616C69676E3D2263656E74D1
:1007C0006572223E3C623E73746174653C2F623EEA
:1007D0003C2F74643E0D0A20202020202020202061
:1007E000203C746420616C69676E3D2263656E74A1
:1007F0006572223E3C623E616374696F6E733C2F8A
:10080000623E3C2F74643E0D0A20202020202020D0
:10081000203C2F74723E0D0A202020202020202012
:100820003C74723E0D0A2020202020202020202011
:100830003C746420616C69676E3D2263656E74650B
:1008400072223E3C623E313C2F623E3C2F74643E3D
:100850000D0A202020202020202020203C7464200D
:10086000616C69676E3D2263656E746572223E3C01
:10087000696D67207372633D222F696D6791222035
:10088000616C743D22818181223E266E6273703BD1
:100890008181813C2F74643E0D0A2020202020207D
:1008A000202020203C746420616C69676E3D2263C7
:1008B000656E746572223E3C6120687265663D22F9
:1008C0002F6F6E31223E6F6E3C2F613E266E62733B
:1008D000703B266E6273703B3C6120687265663DBA
:1008E000222F6F666631223E266E6273703B6F6602
:1008F000663C2F613E3C2F74643E0D0A2020202070
:10090000202020203C2F74723E0D0A202020202021
:100910002020203C74723E0D0A2020202020202020
:100920002020203C746420616C69676E3D22636501
:100930006E746572223E3C623E323C2F623E3C2F1A
:1009400074643E0D0A202020202020202020203CFE
:10095000746420616C69676E3D2263656E746572B4
:10096000223E3C696D67207372633D222F696D677B
:10097000922220616C743D22828282223E266E6227
:1009800073703B8282823C2F74643E0D0A202020CB
:10099000202020202020203C746420616C69676E38
:1009A0003D2263656E746572223E3C61206872650B
:1009B000663D222F6F6E32223E6F6E3C2F613E26C7
:1009C0006E6273703B266E6273703B3C612068728E
:1009D00065663D222F6F666632223E266E62737018
:1009E0003B6F66663C2F613E3C2F74643E0D0A20CF
:1009F000202020202020203C2F74723E0D0A202031
:100A00002020202020203C74723E0D0A202020202F
:100A10002020202020203C746420616C69676E3D9A
:100A20002263656E746572223E3C623E333C2F62E7
:100A30003E3C2F74643E0D0A2020202020202020E0
:100A400020203C746420616C69676E3D2263656E92
:100A5000746572223E3C696D67207372633D222F7C
:100A6000696D67932220616C743D22838383223EEB
:100A7000266E6273703B8383833C2F74643E0D0A41
:100A8000202020202020202020203C746420616C25
:100A900069676E3D2263656E746572223E3C61201B
:100AA000687265663D222F6F6E33223E6F6E3C2F5B
:100AB000613E266E6273703B266E6273703B3C61D2
:100AC00020687265663D222F6F666633223E266E71
:100AD0006273703B6F66663C2F613E3C2F74643ED0
:100AE0000D0A20202020202020203C2F74723E0D53
:100AF0000A20202020202020203C74723E0D0A2055
:100B00002020202020202020203C746420616C695B
:100B1000676E3D2263656E746572223E3C623E34B0
:100B20003C2F623E3C2F74643E0D0A202020202082
:100B300020202020203C746420616C69676E3D2277
:100B400063656E746572223E3C696D6720737263E3
:100B50003D222F696D67942220616C743D2284844C
:100B600084223E266E6273703B8484843C2F7464BE
:100B70003E0D0A202020202020202020203C7464CC
:100B800020616C69676E3D2263656E746572223EFA
:100B90003C6120687265663D222F6F6E34223E6F85
:100BA0006E3C2F613E266E6273703B266E627370E0
:100BB0003B3C6120687265663D222F6F6666342279
:100BC0003E266E6273703B6F66663C2F613E3C2F23
:100BD00074643E0D0A20202020202020203C2F7409
:100BE000723E0D0A20202020202020203C74723EDE
:100BF0000D0A202020202020202020203C7464206A
:100C0000616C69676E3D2263656E746572223E3C5D
:100C1000623E353C2F623E3C2F74643E0D0A20201C
:100C200020202020202020203C746420616C6967F3
:100C30006E3D2263656E746572223E3C696D67206D
:100C40007372633D222F696D67952220616C743D3C
:100C500022858585223E266E6273703B8585853CA4
:100C60002F74643E0D0A20202020202020202020E8
:100C70003C746420616C69676E3D2263656E7465C7
:100C800072223E3C6120687265663D222F6F6E3590
:100C9000223E6F6E3C2F613E266E6273703B266E65
:100CA0006273703B3C6120687265663D222F6F66FF
:100CB0006635223E266E6273703B6F66663C2F611E
:100CC0003E3C2F74643E0D0A20202020202020204E
:100CD0003C2F74723E0D0A20202020202020203C32
:100CE00074723E0D0A202020202020202020203C4D
:100CF000746420616C69676E3D2263656E74657211
:100D0000223E3C623E363C2F623E3C2F74643E0DD8
:100D10000A202020202020202020203C74642061F4
:100D20006C69676E3D2263656E746572223E3C6934
:100D30006D67207372633D222F696D679622206173
:100D40006C743D22868686223E266E6273703B86D8
:100D500086863C2F74643E0D0A202020202020200F
:100D60002020203C746420616C69676E3D226365BD
:100D70006E746572223E3C6120687265663D222F6A
:100D80006F6E36223E6F6E3C2F613E266E62737030
:100D90003B266E6273703B3C6120687265663D2243
:100DA0002F6F666636223E266E6273703B6F6666F4
:100DB0003C2F613E3C2F74643E0D0A2020202020F1
:100DC0002020203C2F74723E0D0A2020202020205D
:100DD00020203C74723E0D0A20202020202020205C
:100DE00020203C746420616C69676E3D2263656EEF
:100DF000746572223E3C623E373C2F623E3C2F744B
:100E0000643E0D0A202020202020202020203C7439
:100E10006420616C69676E3D2263656E7465722241
:100E20003E3C696D67207372633D222F696D679741
:100E30002220616C743D22878787223E266E627372
:100E4000703B8787873C2F74643E0D0A202020204A
:100E50002020202020203C746420616C69676E3D56
:100E60002263656E746572223E3C6120687265661D
:100E70003D222F6F6E37223E6F6E3C2F613E266EF5
:100E80006273703B266E6273703B3C6120687265D2
:100E9000663D222F6F666637223E266E6273703B78
:100EA0006F66663C2F613E3C2F74643E0D0A202025
:100EB0002020202020203C2F74723E0D0A2020206C
:100EC00020202020203C74723E0D0A20202020206B
:100ED00020202020203C746420616C69676E3D22D4
:100EE00063656E746572223E3C623E383C2F623E02
:100EF0003C2F74643E0D0A2020202020202020203A
:100F0000203C746420616C69676E3D2263656E7479
:100F10006572223E3C696D67207372633D222F69C2
:100F20006D67982220616C743D22888888223E2655
:100F30006E6273703B8888883C2F74643E0D0A2073
:100F40002020202020202020203C746420616C6917
:100F5000676E3D2263656E746572223E3C61206857
:100F60007265663D222F6F6E38223E6F6E3C2F6198
:100F70003E266E6273703B266E6273703B3C61204E
:100F8000687265663D222F6F666638223E266E6265
:100F900073703B6F66663C2F613E3C2F74643E0D60
:100FA0000A20202020202020203C2F74723E0D0A91
:100FB0002020202020203C2F7461626C653E0D0AA9
:100FC0002020202020203C62723E3C62723E0D0AAE
:100FD0002020202020203C6120687265663D222F61
:100FE000223E726566726573683C2F613E0D0A2071
:100FF000203C2F626F64793E0D0A3C2F68746D6C43
:101000003E0D0A00485454502F312E3020343034D5
:10101000204E6F7420466F756E640D0A53657276AC
:1010200065723A2038426974416D45746865726E24
:101030006574202841544D4547413132382920629A
:1010400079204343432D41432E64650D0A436F6E5F
:101050006E656374696F6E3A20636C6F73650D0A19
:10106000436F6E74656E742D547970653A207465A3
:1010700078742F68746D6C0D0A0D0A3C68746D6C81
:101080003E0D0A20203C686561643E3C7469746CC6
:10109000653E38426974416D45746865726E657469
:1010A000202D20343034204E6F7420466F756E64CE
:1010B0003C2F7469746C653E3C2F686561643E0D1D
:1010C0000A20203C626F64793E0D0A202020203CDB
:1010D00068313E38426974416D45746865726E6569
:1010E00074202D20343034204E6F7420466F756E7E
:1010F000643C2F68313E0D0A202020205468652072
:101100007265717565737465642055524C20776102
:1011100073206E6F7420666F756E64206F6E20741E
:10112000686973207365727665722E3C62723E0D3B
:101130000A20203C2F626F64793E0D0A3C2F6874B0
:101140006D6C3E0D0A00485454502F312E3020341F
:1011500030302042616420526571756573740D0AE8
:101160005365727665723A2038426974416D4574F0
:101170006865726E6574202841544D45474131328F
:101180003829206279204343432D41432E64650D65
:101190000A436F6E6E656374696F6E3A20636C6F9D
:1011A00073650D0A436F6E74656E742D54797065A6
:1011B0003A20746578742F68746D6C0D0A0D0A3CC2
:1011C00068746D6C3E0D0A20203C686561643E3C8D
:1011D0007469746C653E38426974416D4574686524
:1011E000726E6574202D20343030204261642052AC
:1011F0006571756573743C2F7469746C653E3C2F22
:10120000686561643E0D0A20203C626F64793E0D82
:101210000A202020203C68313E38426974416D45E7
:10122000746865726E6574202D2034303020426100
:101230006420526571756573743C2F68313E0D0AE8
:1012400020202020596F75722062726F777365724B
:101250002073656E742061207265717565737420EA
:10126000746861742074686973207365727665723E
:1012700020636F756C64206E6F7420756E64657288
:101280007374616E642E3C62723E0D0A20203C2F06
:10129000626F64793E0D0A3C2F68746D6C3E0D0AD6
:1012A000000011241FBECFEFD0E1DEBFCDBF11E0A3
:1012B000A0E0B1E0E2EDF5E600E00BBF02C0079070
:1012C0000D92A63AB107D9F717E0A6EAB1E001C03E
:1012D0001D92A737B107E1F70C9470090C94000038
:1012E000CFEFD0E1DEBFCDBFA89588E190E02AE046
:1012F0000FB6F894A89581BD0FBE21BDA8950E9498
:10130000DF2C0E949C090E946C150E9425180E94E7
:10131000E8190E94731B0E94CC1E0E9406200E94A6
:10132000D12C0E94F70F7894A8950E9439110E9441
:10133000F0180E94D51EF8CFE3ECF1E08BE01082AC
:101340003C96815087FFFBCF0895CF93DF93CDB7B5
:10135000DEB7AA970FB6F894DEBF0FBECDBFFC0173
:1013600020E031E02F87388B88E090E0898B9A8BE2
:1013700086E08B8B84E08C8B2D8B3E8B80911001D3
:101380008F8B80911101888F80911201898F8091BC
:1013900013018A8F809114018B8F809115018C8F9E
:1013A00080910C018D8F80910D018E8F80910E01A7
:1013B0008F8F80910F0188A39FEF99A39AA39BA37E
:1013C0009CA39DA39EA380818FA3818188A78281F6
:1013D00089A783818AA799839A839B839C839D8312
:1013E0009E8388E096E08D879E876AE270E0CE015A
:1013F00001960E941D12AA960FB6F894DEBF0FBE8A
:10140000CDBFDF91CF910895FF920F931F93CF939C
:10141000DF930BEC11E0E80128978BE0F82E888130
:10142000282F332720FF15C099819F5F998321FFC3
:1014300003C0973970F002C0933310F0188209C0CE
:10144000892F992787709070892B19F4C8010E9401
:10145000A509FA942C96045F1F4FF7FEE0CFDF91A9
:10146000CF911F910F91FF9008951F93CF93DF931A
:10147000CDB7DEB7AA970FB6F894DEBF0FBECDBFCB
:10148000DC016A32710508F42FC1FD01868597855C
:101490008050914009F028C1FD0180899189089709
:1014A00009F022C18289863009F01EC18389843007
:1014B00009F01AC166896F3F81F487898F3F69F40B
:1014C000808D8F3F51F4818D8F3F39F4828D8F3F16
:1014D00021F4838D8F3F09F407C1FD0124893589EB
:1014E000F1E020303F0709F061C0FD0116A18091B5
:1014F0000C01181709F05AC077A180910D017817D7
:1015000009F054C050A580910E01581709F04EC043
:1015100041A580910F01481709F048C02F87388BEB
:1015200088E090E0898B9A8B86E08B8B84E08C8BB3
:1015300080E092E08D8B9E8B809110018F8B80914B
:101540001101888F80911201898F809113018A8FF8
:10155000809114018B8F809115018C8F1D8F7E8F50
:101560005F8F48A369A357895AA3408D4BA3318D40
:101570003CA3228D2DA3938D9EA3848D8FA3858D57
:1015800088A7868D89A7878D8AA769835A834B830D
:101590003C832D839E8388E096E08D879E876AE258
:1015A00070E0CE0101960E941D129EC02050324074
:1015B00009F09AC0FD0190A180911001981709F0DF
:1015C00093C091A180911101981709F08DC092A14B
:1015D00080911201981709F087C093A1809113019F
:1015E000981709F081C094A180911401981709F00F
:1015F0007BC095A180911501981709F075C096A13F
:1016000080910C01981709F06FC097A180910D018E
:10161000981709F069C090A580910E01981709F0FC
:1016200063C091A580910F01981709F05DC040E05B
:1016300023EC31E0F901808180FF18C0FD01948D19
:10164000F9018085981791F4FD01958DF901818547
:10165000981761F4FD01968DF9018285981731F490
:10166000FD01978DF9018385981729F04F5F245F5D
:101670003F4F4C30F8F24C30B8F5242F33278CE034
:1016800090E0289FB001299F700D389F700D1124A4
:101690009B012D533E4F83E0F90180831182FD01B0
:1016A0008689F9018283FD018789F9018383FD0120
:1016B000808DF9018483FD01818DF9018583FD0110
:1016C000828DF9018683FD01838DF90187838CE08A
:1016D000489F90011124C9018B539E4FBC01C90141
:1016E00085539E4F0E949217AA960FB6F894DEBFBC
:1016F0000FBECDBFDF91CF911F9108950F931F9320
:10170000CF93DF93DC012C9180910C01281789F491
:10171000ED01998180910D01981759F49A8180917A
:101720000E01981731F49B8180910F01981709F4ED
:1017300080C040E0E3ECF1E0808180FF10C0808554
:10174000281769F4ED0199818185981741F49A81F0
:101750008285981721F49B818385981721F04F5F2C
:101760003C964C3048F34C3008F43FC040E0E3EC8A
:10177000F1E080813C9680FF03C04F5F4C30C8F39E
:101780004C30D0F040E021E00CE010E0C0EDD1E0C2
:10179000842F9927809FF001819FF00D909FF00D7D
:1017A0001124ED53FE4F98812C968181891708F4FE
:1017B000422F2F5F2C3060F3242F33278CE090E0F2
:1017C000289FF001299FF00D389FF00D1124ED5353
:1017D000FE4F81E0808311828C918087ED018981A9
:1017E00081878A8182878B818387842F99272CE048
:1017F00030E0829FF001839FF00D929FF00D112445
:10180000ED53FE4F808181FF11C08281DB018C93FB
:101810008381EB01898384818A8385818B8386819F
:101820008C8387818D8380E090E005C0CD010E948C
:10183000A50981E090E0DF91CF911F910F9108956C
:10184000CF93DF93EC01FB01CA01AC016627772738
:10185000C901AA27BB27480F591F6A1F7B1FE23007
:10186000F10580F029913991832F9927322F222772
:10187000822B932BAA27BB27480F591F6A1F7B1F58
:101880003297EDCFEF2B51F088819927982F882739
:10189000AA27BB27480F591F6A1F7B1FDB01CA01FC
:1018A000A070B070AB0166277727480F591F6A1FD9
:1018B0007B1FDB01CA01A070B0709B014427552734
:1018C000820F931FA41FB51F80959095DF91CF9134
:1018D00008958F929F92AF92BF92CF92DF92EF9234
:1018E000FF920F931F93CF93DF93CDB7DEB760972F
:1018F0000FB6F894DEBF0FBECDBF6C01662319F49E
:1019000080E090E061C3623008F45CC3FC01808138
:1019100099278032910509F41EC28132910594F411
:101920008031910509F476C0813191051CF4892B31
:10193000E9F048C38131910509F4E4C0429709F404
:1019400092C140C38033910509F4C1C2813391052E
:1019500024F4819709F44AC235C38034910509F40F
:1019600001C38134910509F404C32CC3683009F024
:1019700002C3F6012181922F92959F7084E6989F71
:10198000A001112433272F703070C90103E0880FA4
:10199000991F0A95E1F7820F931F820F931F642FFF
:1019A000680F828182958F70680F828199278F706E
:1019B000907024E630E0829FA001839F500D929F9B
:1019C000500D11242381922F92959F708AE0989F49
:1019D000C0011124942F980F2F70920FF89482E079
:1019E000809310018CEC8093110180EC80931201A4
:1019F0008CEA8093130160931401909315017894FD
:101A00008091B80181608093B801F8940E94AD1A6A
:101A10007894D4C26E3009F0AEC2F6019181892F5C
:101A200082958F70B4E68B9FA0011124292F332754
:101A30002F703070C90113E0880F991F1A95E1F7D4
:101A4000820F931F820F931F742F780F82818295CC
:101A50008F70780F828199278F70907004E610E064
:101A6000809FA001819F500D909F500D11242381D4
:101A7000822F82958F70AAE08A9FC0011124642F63
:101A8000680F2F70620F9481892F82958F708B9FC2
:101A9000A0011124292F33272F703070C901B3E022
:101AA000880F991FBA95E1F7820F931F820F931F3A
:101AB000342F380F9581892F82958F70380F892F99
:101AC00099278F709070809FA001819F500D909FEB
:101AD000500D11242681822F82958F708A9FC0011C
:101AE0001124840F2F70820FF89470930C0160936F
:101AF0000D0130930E0180930F0178948091B8010D
:101B000082605AC26E3009F036C2F6019181892F87
:101B100082958F70A4E68A9FA0011124292F332774
:101B20002F703070C90163E0880F991F6A95E1F743
:101B3000820F931F820F931F942F980F828182959B
:101B40008F70E92EE80E828199278F70907064E67D
:101B500070E0869FA001879F500D969F500D112425
:101B60002381822F82958F70BAE08B9FC001112450
:101B7000840F2F70F82EF20E9481892F82958F702A
:101B80008A9FA0011124292F33272F703070C9019B
:101B900053E0880F991F5A95E1F7820F931F820F28
:101BA000931F242F280F9581892F82958F70022FE4
:101BB000080F892F99278F709070869FA001879FAB
:101BC000500D969F500D11242681822F82958F7083
:101BD0008B9FC0011124840F2F70820F282F332771
:101BE000122F8E2D9927AA27BB27782F66275527D6
:101BF00044278F2D9927AA27BB27DC0199278827FF
:101C0000482B592B6A2B7B2B802F9927AA27BB2780
:101C1000BA2FA92F982F8827482B592B6A2B7B2B5B
:101C2000822F9927AA27BB27482B592B6A2B7B2B5E
:101C300077232CF4440F551F661F771FF9CF4115EA
:101C400051056105710509F096C1F894E09208010B
:101C5000F092090100930A0110930B01789480918E
:101C6000B8018460A9C16E3009F085C1F601918187
:101C7000892F82958F70B4E68B9FA0011124292FA4
:101C800033272F703070C90163E0880F991F6A9560
:101C9000E1F7820F931F820F931F742F780F8281B9
:101CA00082958F70780F828199278F70907004E6EB
:101CB00010E0809FA001819F500D909F500D112436
:101CC0002381822F82958F70AAE08A9FC001112400
:101CD000642F680F2F70620F9481892F82958F7007
:101CE0008B9FA0011124292F33272F703070C90139
:101CF00053E0880F991F5A95E1F7820F931F820FC7
:101D0000931F342F380F9581892F82958F70380F4C
:101D1000892F99278F709070809FA001819F500D0F
:101D2000909F500D11242681822F82958F708A9F5B
:101D3000C0011124840F2F70820FF8947093040156
:101D40006093050130930601809307017894809198
:101D5000B801886031C1673009F00DC1F6012281F8
:101D6000922F92959F7084E6989FB001112433279B
:101D70002F703070C90113E0880F991F1A95E1F791
:101D8000820F931F820F931F680F791FA1818A2FE3
:101D900082958F70282F332780E197E2289FA0013A
:101DA000299F500D389F500D11248A2F99278F702D
:101DB000907028EE33E0829FF001839FF00D929F98
:101DC000F00D11244E0F5F1F640F751FF601838104
:101DD00082958F70680F711DF89470930301609362
:101DE000020178948091B8018061E6C0623309F005
:101DF000C2C020E042E0BE016F5F7F4FB1E0AB2E7A
:101E0000B12CA4E68A2EF4E6EF2EF12CEAE09E2E09
:101E1000DB01A20FB11D842F992781709070342FA0
:101E20003695122F1F5F042F0D5F8A159B0509F150
:101E3000F601E30FF11D9081892F82958F70889DA7
:101E4000A0011124292F33272F703070C90153E0CE
:101E5000880F991F5A95E1F7820F931F820F931FE6
:101E6000942F980F818182958F70980F892F9927D1
:101E700019C0F601E30FF11D808199278F709070D2
:101E80008E9DA0018F9D500D9E9D500D112421818E
:101E9000822F82958F70899DC0011124840F2F702D
:101EA000820F99278C93212F402F103108F4B0CF47
:101EB000F894A7EAB1E0FB012FE081918D932150C6
:101EC00027FFFBCF78948091B801806275C067309E
:101ED00009F051C0F6012281922F92959F7084E6FD
:101EE000989FB001112433272F703070C90143E04F
:101EF000880F991F4A95E1F7820F931F820F931F56
:101F0000680F791FA1818A2F82958F70282F332720
:101F100080E197E2289FA001299F500D389F500D26
:101F200011248A2F99278F70907028EE33E0829FBA
:101F3000F001839FF00D929FF00D11244E0F5F1F53
:101F4000640F751FF601838182958F70680F711D74
:101F5000F894709301016093000178948091B80126
:101F600080642AC0623039F40E94451A8093A60129
:101F700020C06A3019F08FEF90E022C090E031E08D
:101F8000F601319696952191822F82958F7082303D
:101F900090F7813009F490689695822F8F70823087
:101FA00050F7813009F490683F5F353058F39093D3
:101FB000A6018091B80180688093B80180E090E02C
:101FC000992702C08FEF90E060960FB6F894DEBFBD
:101FD0000FBECDBFDF91CF911F910F91FF90EF907A
:101FE000DF90CF90BF90AF909F908F900895E0E1E9
:101FF000F1E046E01FBA1EBA30E0E09A2DB38EB38E
:102000009FB301969FBB8EBBE09A8DB328278EB3FA
:102010009FB301969FBB8EBB2F3F89F43F5F363045
:1020200060F31FBA1EBAE09A8DB381938EB39FB34B
:1020300002969FBB8EBB4150B1F70E94AD1A4CE097
:1020400050E0ECE0F1E064E05FBB4EBB30E0E09AD2
:102050002DB38EB39FB301969FBB8EBBE09A8DB319
:1020600028278EB39FB301969FBB8EBB2F3F79F479
:102070003F5F343060F35FBB4EBBE09A8DB381931A
:102080008EB39FB302969FBB8EBB6150B1F744E104
:1020900050E0E8E0F1E064E05FBB4EBB30E0E09A86
:1020A0002DB38EB39FB301969FBB8EBBE09A8DB3C9
:1020B00028278EB39FB301969FBB8EBB2F3F79F429
:1020C0003F5F343060F35FBB4EBBE09A8DB38193CA
:1020D0008EB39FB302969FBB8EBB6150B1F74CE1AC
:1020E00050E0E4E0F1E064E05FBB4EBB30E0E09A3A
:1020F0002DB38EB39FB301969FBB8EBBE09A8DB379
:1021000028278EB39FB301969FBB8EBB2F3F79F4D8
:102110003F5F343060F35FBB4EBBE09A8DB3819379
:102120008EB39FB302969FBB8EBB6150B1F744E262
:1021300050E0E2E0F1E062E05FBB4EBB30E0E09AED
:102140002DB38EB39FB301969FBB8EBBE09A8DB328
:1021500028278EB39FB301969FBB8EBB2F3F79F488
:102160003F5F323060F35FBB4EBBE09A8DB381932B
:102170008EB39FB302969FBB8EBB6150B1F748E20E
:1021800050E0E7EAF1E060E15FBB4EBB30E0E09A8F
:102190002DB38EB39FB301969FBB8EBBE09A8DB3D8
:1021A00028278EB39FB301969FBB8EBB2F3F79F438
:1021B0003F5F303160F35FBB4EBBE09A8DB38193DC
:1021C0008EB39FB302969FBB8EBB6150B1F748E4BC
:1021D00050E0E0E0F1E062E05FBB4EBB30E0E09A4F
:1021E0002DB38EB39FB301969FBB8EBBE09A8DB388
:1021F00028278EB39FB301969FBB8EBB2F3F79F4E8
:102200003F5F323060F35FBB4EBBE09A8DB381938A
:102210008EB39FB302969FBB8EBB6150B1F74CE467
:1022200050E0E6EAF1E031E05FBB4EBBE09A2DB34F
:102230008EB39FB301969FBB8EBBE09A8DB32827C8
:102240008EB39FB301969FBB8EBB2F3F81F45FBBC4
:102250004EBBE09A8DB381938EB39FB302969FBB22
:102260008EBB3150B1F78091A6010E94491A0895A2
:1022700008958091B7019927AC014170507080FD9D
:1022800091C02091B801822F992780FF0FC02E7F27
:102290002093B80180E191E090935502809354021D
:1022A000509357024093560286E012C081FF14C03B
:1022B0002D7F2093B8018CE091E09093550280939C
:1022C00054028CE090E0909357028093560284E091
:1022D0008093530281E064C082FF0CC02B7F209367
:1022E000B80188E091E0909355028093540284E114
:1022F00090E0E9CF83FF0CC0277F2093B80184E0F2
:1023000091E090935502809354028CE190E0DBCFF2
:1023100084FF0CC02F7E2093B80182E091E090935F
:1023200055028093540284E290E020C085FF11C0E2
:102330002F7D2093B80187EA91E090935502809316
:10234000540288E290E0909357028093560280E115
:10235000BFCF86FF11C02F7B2093B80180E091E0B2
:10236000909355028093540288E490E09093570232
:102370008093560282E0ACCF27FF48C02F7720938E
:10238000B80186EA91E090935502809354028CE460
:1023900090E0909357028093560281E0809353021D
:1023A0008093B701E19932C0F894809156029091E0
:1023B00057029C01019690935702809356023FBBAF
:1023C0002EBB9091B701E0915402F091550291FF1C
:1023D00012C081918095F0935502E09354028DBB19
:1023E00080915302815080935302882331F49E7F61
:1023F0009093B70102C080818DBB8091B70192E0BC
:1024000089278093B701E29AE19A78940895089514
:10241000FC016E30710578F08485958588309105D2
:1024200039F08850964039F4CF010E94350A08955A
:10243000CF010E94E01508950895FC016E307105EA
:10244000A8F080911001868380911101878380918B
:102450001201808780911301818780911401828706
:10246000809115018387CF010E94AE1B08950895C6
:10247000CF93DF93EC018E89833069F443E050E021
:1024800060E271E0CE0106960E945E31892B19F45C
:1024900081E08F8B01C01F8ADF91CF9108950F9348
:1024A0001F93CF93DF93EC011E89113061F441E05B
:1024B00050E064E271E006960E945E31892B09F0DB
:1024C00040C0198F3FC0143081F443E050E066E211
:1024D00071E006960E945E31892B99F589858133DA
:1024E00080F1893370F58F522AC0153051F544E0E0
:1024F00050E06AE271E006960E945E31892B39F461
:102500008A85813320F0893310F4875218C08E01F8
:102510000A5F1F4F45E050E06FE271E0C8010E9482
:102520005E31892B11F482E10AC045E050E065E399
:1025300071E0C8010E945E31892B19F483E1898F13
:1025400001C0198EDF91CF911F910F910895CF9304
:10255000DF93EC018F89813009F06AC0698D862F85
:102560009927823091057CF08A3091051CF04297C2
:1025700054F403C0615081E002C0695080E00E94C1
:10258000071A81E0898F898D992782319105D1F0D1
:10259000833191051CF4019721F039C0439719F15B
:1025A00036C0888D882339F086E596E08A8F9B8F28
:1025B0008DEA99E04DC086EE95E08A8F9B8F8DE184
:1025C0009AE046C0888D882339F08AE993E08A8FA3
:1025D0009B8F8BE492E017C08AE293E08A8F9B8FF7
:1025E0008BEB92E010C0888D882339F08CEF90E05F
:1025F0008A8F9B8F8DE292E006C08CE890E08A8FF4
:102600009B8F8DE992E08C8F9D8F1E8E25C0888DCB
:10261000882339F08BE790E18A8F9B8F8AEC90E0DA
:1026200017C084E090E18A8F9B8F81E491E010C015
:10263000888D882339F08FEB91E18A8F9B8F81EE13
:1026400090E006C086E491E18A8F9B8F8AE591E055
:102650008C8F9D8F81E08E8FDF91CF910895CF93E6
:10266000DF93EB01282F3327213831057CF12938FE
:10267000310534F0215930402830310538F518C083
:10268000433020F180580E94EE19882339F08FE4FE
:102690009EE48883998382E090E01AC083E0EBE3B4
:1026A000F1E0019009928A95E1F783E090E010C093
:1026B000442361F080590E94EE19882311F081E3D0
:1026C00001C080E3888381E090E002C080E090E078
:1026D000DF91CF910895282F90E0E8E5F2E0808126
:1026E0007F96821719F09F5F9430C8F3943060F0A2
:1026F00090E0E8E5F2E080817F968F3F19F09F5FE0
:102700009430C8F3943068F48FE1989FF00111245D
:10271000E85AFD4F2083118212821382148215829F
:10272000168A08950895282F90E0E8E5F2E0808168
:102730007F96821719F09F5F9430C8F3943040F46D
:102740008FE1989FF0011124E85AFD4F8FEF8083AD
:10275000089508956F927F928F929F92AF92BF9249
:10276000CF92DF92EF92FF920F931F93CF93DF935D
:10277000CDB7DEB761970FB6F894DEBF0FBECDBF01
:10278000A82F490190E0E8E5F2E080817F968A1762
:1027900019F09F5F9430C8F39430D0F48FE1989F84
:1027A0006001112488E592E0C80ED91EF6018581EA
:1027B000833019F000E010E07AC0F601248D358DE9
:1027C000C901AA27BB27481759076A077B0718F0D2
:1027D0000FEF1FEF6CC0C901841B950B58018017C8
:1027E000910708F45C01A114B10409F45FC0EE2460
:1027F000AE2D9E2DF601028D138D040F151FF801CD
:10280000F490F601868D8823F1F0F7FE1CC0EF2CC2
:1028100040E1BE016F5F7F4F8F2DA98B0E942F1368
:10282000A82FA80141505040F601228D338D99897F
:102830002417350740F4FA0184918F1521F49F5F26
:1028400041505040F5CFA114B10481F13501F80198
:10285000F490F601868D8823D9F0F7FE19C0EF14A5
:1028600051F0EF2C40E1BE016F5F7F4F8F2D0E9432
:102870002F13A82F90E09A1738F4FE013196E90F34
:10288000F11D9F5F808101C080E2F401808303C05D
:10289000EE24F401F0820F5F1F4F0894811C911CFD
:1028A0000894610871086114710489F68501C801F2
:1028B00061960FB6F894DEBF0FBECDBFDF91CF910A
:1028C0001F910F91FF90EF90DF90CF90BF90AF904E
:1028D0009F908F907F906F9008950895AF92BF92D0
:1028E000CF92DF92EF92FF920F931F93CF93DF93DC
:1028F000A82F6901580190E0E8E5F2E080817F9619
:102900008A1719F09F5F9430C8F3943038F0C701EC
:1029100021E08030920708F0D4C0D1C08FE1989FA9
:10292000E0011124C85ADD4F89819A81AB81BC81B5
:1029300084179507A607B70761F088810E94BE2B10
:102940008FEF8883C701A1E080309A0708F0B9C0F3
:10295000B6C0A114B10409F4ADC09E89903140F411
:10296000FE01E90FF11DD6018C9186839F5F9E8B3E
:102970008D8199278130910559F1823091051CF4A0
:10298000892B49F085C08230910509F43FC0039737
:1029900009F47DC07DC0F60180818D3011F08A3050
:1029A00051F48E8981508E8BCE010E94381281E0C5
:1029B000888F898F65C0803219F0893009F068C02E
:1029C0008E8981508E8BCE010E94381281E01CC00E
:1029D000D6018C918D3011F08A3049F48E89815066
:1029E0008E8BCE010E944F1281E0888F49C08032C9
:1029F00019F0893009F04CC08E8981508E8BCE0140
:102A00000E944F12188E82E08D8341C0F6018081B2
:102A10008D3011F08A30D9F51E891230A9F442E0C8
:102A200050E06FE371E0CE0106960E947830892B6A
:102A300039F142E050E062E471E0CE0106960E9476
:102A40007830892BE9F00DC0133059F443E050E0A1
:102A500065E471E0CE0106960E947830892B81F002
:102A600002C0133059F443E050E069E471E0CE0154
:102A700006960E947830892B19F00AC0143041F470
:102A800083E08D831E8ACE010E94A71201C01E8A98
:102A90000894C11CD11C0894A108B10889819A81AD
:102AA000AB81BC810196A11DB11D89839A83AB8343
:102AB000BC834FCFC701F1E080309F0710F480E066
:102AC00091E0DF91CF911F910F91FF90EF90DF90F8
:102AD000CF90BF90AF9008959FEFE8E5F2E083E0DC
:102AE00090837F96815087FFFBCF0895CF92DF922E
:102AF000EF92FF920F931F93CF93DF93EC018B0123
:102B00006632710508F440C07EEDE72E7FEFF72EA8
:102B1000E00EF11E62E2C62ED12CC80ED91E20E0B6
:102B200030E0A901B701C6010E94200CAC01892B3D
:102B300059F58AA1883041F50A32110528F18BA197
:102B4000882311F58AA38A8D8E8F8B8D8F8F8C8D24
:102B500088A38D8D89A306321105B0F04CA35DA327
:102B60009A01B701C6010E94200C9C01892F992768
:102B7000322F2227822B932B8CA39DA381E08F8B56
:102B8000B801CE010E94F516DF91CF911F910F91F0
:102B9000FF90EF90DF90CF900895EDE4F1E023E017
:102BA00084819581892B39F086818F5F8683833379
:102BB00010F0148215822150379627FFF1CF089527
:102BC000CF92DF92EF92FF920F931F93CF93DF93F9
:102BD0008C016B016232710508F4FEC0E8018E853C
:102BE000853409F0F9C08E8DF0900C018F1509F035
:102BF000F3C08F8D20910D01821709F0EDC088A1DF
:102C000030910E01831709F0E7C089A140910F01AF
:102C1000841709F0E1C05A8D503E08F0DDC05F37DF
:102C200009F4DAC0552351F48B8D882339F48C8D47
:102C3000882321F48D8D882309F4CEC0E09108010A
:102C4000952F9E238F2D8E23981709F072C0E801CF
:102C5000EB8CF09109018E2D8F232F23821709F021
:102C600068C06C8DA0910A01862F8A233A238317AE
:102C700009F05FC07D8DB0910B01872F8B234B2313
:102C8000841709F056C0252F33278E2F992780955A
:102C9000909528233923232BF9F42E2D33278F2FBA
:102CA00099278095909528233923232BA9F4262F43
:102CB00033278A2F99278095909528233923232B12
:102CC00059F4272F33278B2F992780959095282308
:102CD0003923232B09F480C0252F33278E2F9927E2
:102CE00080959095282339232F3F310511F52E2DFE
:102CF00033278F2F992780959095282339232F3FAD
:102D00003105B9F4262F33278A2F9927809590957E
:102D1000282339232F3F310561F4272F33278B2FA9
:102D2000992780959095282339232F3F310509F461
:102D300053C0F801828D8F1581F4938D80910D0120
:102D4000981759F4948D80910E01981731F4958D50
:102D500080910F01981709F43FC0E8018C899D8983
:102D6000492F5527982F8827482B592B5F7B4115D2
:102D7000510591F588899989C92FDD27982F8827D2
:102D8000C82BD92B2E96CC16DD0630F19A0164E1C2
:102D900070E0C8010E960E94200C892BE9F4F8011E
:102DA000878999278630910571F0873091051CF449
:102DB000019721F011C0419759F00EC0BE01C80122
:102DC0000E94761509C0BE01C8010E942B2404C0D0
:102DD000BE01C8010E94482DDF91CF911F910F9134
:102DE000FF90EF90DF90CF900895EF92FF920F93B6
:102DF0001F93CF93DF93EC017B016232710508F4DE
:102E00008AC085E48E871F869B012E503040832F19
:102E10009927322F2227822B932B888B998B1A8A02
:102E20001B8A1C8A1D8A80E48E8B188E198E8091D5
:102E30000C018A8F80910D018B8F80910E018C8FF8
:102E400080910F018D8F20E030E0A90164E170E0F6
:102E5000CE010E960E94200C9C01892F9927322FBB
:102E60002227822B932B888F998F9E8D209108018A
:102E7000922380910C0182239817F9F48F8D209171
:102E80000901822390910D0192238917B1F488A141
:102E900020910A01822390910E019223891769F4EF
:102EA00089A120910B01822390910F019223891710
:102EB00021F4BE01CE014E9603C0BE0184E091E034
:102EC0000E947E0B8823A9F488E090E08C879D8780
:102ED000B701CE010E941D121EC0A701BE01F8015C
:102EE000808191810E948530F801E482F58216820A
:102EF00012C020E00DE411E0F80184819581892B56
:102F000029F482819381E816F90638F32F5F095F6F
:102F10001F4F243088F3DF91CF911F910F91FF90C5
:102F2000EF900895AF92BF92DF92EF92FF920F93CE
:102F30001F93CF93DF938C015B018DE4E82E81E03A
:102F4000F82EC3E0DC2EE7018C819D81892B09F4EA
:102F50006BC0E881F981668D80910801262F2823B6
:102F600090910C019823291769F5578D80910901DB
:102F7000252F282390910D019823291719F540A199
:102F800080910A01242F282390910E01982329175C
:102F9000C9F431A180910B01232F282390910F01B7
:102FA0009823291779F4D8018C916817E9F5E8017D
:102FB00089815817C9F58A814817B1F58B8138176F
:102FC00099F516C090910401D8018C91981761F57C
:102FD00090910501E8018981981731F590910601DA
:102FE0008A81981709F5909107018B819817E1F470
:102FF00088E090E084879587D5018C918083E501F6
:10300000898181838A8182838B8183838C8184837C
:103010008D818583F70164817581808191810E9412
:103020001D12E7011C821D82DA94E7E0F0E0EE0E4B
:10303000FF1ED7FE88CFDF91CF911F910F91FF9098
:10304000EF90DF90BF90AF900895BB98C39ABC9863
:10305000C49A17981F9A12981A9ABD98C59AB89848
:10306000C09A13981B9ABE98C69ABA98C29A159895
:103070001D9ABF98C79A16981E9A80916400816025
:10308000809364008091640082608093640084E097
:10309000E8E5F5E011921192815087FFFBCF109285
:1030A000550510925405109257051092560510922E
:1030B0006405109263058FEF80936205809165002F
:1030C0008E7F80936500809165008D7F8093650081
:1030D0000895CF93DF93C0E0D0E0B39902C0C1E080
:1030E000D0E0B49BC2600F9BC4600A9BC860B59BD4
:1030F000C061B09BC0620B9BC064B69BC068B29BB2
:10310000D1600D9BD260B79BD4600E9BD86080913C
:103110005805909159058C179D0721F08091C001A9
:103120000E944F1A4FEF5FEF60E070E024E0A0E6EE
:10313000B5E08D919C911197482359238D919C91D5
:103140001197682B792BFD013297808191818D93A6
:103150009C932150DF0169F74C235D236C2B7D2B61
:10316000D0935905C09358052091540530915505C9
:10317000209530952423352380915605909157054D
:10318000822B932B9093570580935605CB01809506
:10319000909520915405309155052823392380912D
:1031A000630590916405822B932B90936405809323
:1031B00063058091540590915505842B952B909330
:1031C00055058093540580915405909155058623AB
:1031D00097239093550580935405DF91CF910895DF
:1031E0001F93CF93DF938091560590915705892FB8
:1031F00099278695869580FF1CC0809156059091F1
:1032000057059B7F909357058093560580916205E3
:103210008695813230F0109262058091650082605F
:1032200006C08FEF80936205809165008D7F80934B
:10323000650090916205892F8695813208F445C01A
:1032400011E0C2E0D0E080915605909157058C23A3
:103250009D23892B99F09E012095309580915605EC
:103260009091570582239323909357058093560599
:10327000F894612F8FEF0E94071A78941F5FCC0F8C
:10328000DD1F193000F3809156059091570580FF9E
:1032900009C080915605909157058E7F90935705F0
:1032A000809356058091560590915705892F99274F
:1032B000869580FF43C080915605909157059D7F6C
:1032C000909357058093560539C010E0C1E0D0E0D7
:1032D000BE01492F512F80915605909157058C239F
:1032E0009D23892B19F19E012095309580915605DB
:1032F0009091570582239323909357058093560509
:10330000E42FE695E03290F4842F99278170907035
:10331000FF278617970721F0EB59FA4F508305C016
:10332000EB59FA4F8081812B80834F5F1F5F505F85
:10333000CC0FDD1F1A3078F240936205809156055C
:1033400090915705892F992786958695869580FFB8
:1033500022C08091560590915705977F909357050D
:103360008093560560916205862F8695813298F488
:1033700085E695E00E94690C882329F48091650018
:103380008160809365008FEF809362058091650076
:103390008D7F809365008091630590916405892FEE
:1033A000992786958695869580FF0EC08091630546
:1033B00090916405977F9093640580936305809155
:1033C00065008E7F80936500DF91CF911F910895F6
:1033D0008FEF81BB8091B90182BB0895982F8150F6
:1033E000883018F080E090E008958091B901282F8E
:1033F0003327892F9927019702C0359527958A95FC
:10340000E2F7822F99278170907008950895982F80
:10341000862F81508830B8F5992399F4262F3327C9
:103420002150304081E090E002C0880F991F2A951A
:10343000E2F7982F90958091B90189238093B90183
:103440001FC0262F332719166CF42150304081E01D
:1034500090E002C0880F991F2A95E2F72091B901E8
:10346000282B0CC02150304081E090E002C0880F32
:10347000991F2A95E2F72091B90128272093B901D5
:103480008091B90182BB089508958091B90199276F
:1034900008958093B9018091B90182BB089520916C
:1034A000BA013091BB014091BC015091BD01220F86
:1034B000331F441F551F9927AA27BB2728273927C1
:1034C0004A275B272093BA013093BB014093BC018C
:1034D0005093BD01809169018F5F80936901809154
:1034E0006901803270F0109269018091BA01909167
:1034F000BB01A091BC01B091BD01BC01CD010E94F6
:103500005331089508950F931F93CF938C01C62FC5
:10351000C33078F00E94EF3022E0F80161938F0110
:10352000672F782F892F9927215027FFF6CFC35077
:10353000EFCFCC2371F00E94EF30CC2351F02C2F31
:10354000F80161938F01672F782F892F99272150D8
:10355000B9F7CF911F910F9108958FEF8ABB80E645
:1035600085BB81E28BBBAE980000AE9A93E600006B
:10357000915097FFFCCF8FEF8ABB8EE685BB88E525
:103580008BBBAE980000AE9A8FEF8ABB8AE685BBF4
:103590001BBAAE980000AE9A8FEF8ABB8BE685BB54
:1035A0001BBAAE980000AE9A8FEF8ABB8CE685BB43
:1035B00084E08BBBAE980000AE9A8FEF8ABB84E6A6
:1035C00085BB86E48BBBAE980000AE9A8FEF8ABBBA
:1035D0008DE685BB82E08BBBAE980000AE9A8FEF84
:1035E0008ABB81E685BB86E48BBBAE980000AE9AB1
:1035F0008FEF8ABB83E685BB86E48BBBAE98000069
:10360000AE9A8FEF8ABB82E685BB80E68BBBAE9815
:103610000000AE9A8FEF8ABB80E685BB81E68BBB4C
:10362000AE980000AE9A93E60000915097FFFCCF51
:103630008FEF8ABB87E685BB86E48BBBAE98000024
:10364000AE9A90E02FEFE0E1F1E02ABB9F5F892F77
:103650008F71806685BB81918BBBAE980000AE9A5E
:103660009050963090F38FEF8ABB80E685BB81E265
:103670008BBBAE980000AE9A8FEF8ABB8EE685BBFF
:1036800088E58BBBAE980000AE9A8FEF8ABB80E6D0
:1036900085BB82E28BBBAE980000AE9A9FEF9ABBCF
:1036A00087E685BB9BBBAE980000AE9A8FEF8ABBC6
:1036B0008FE685BB81E18BBBAE980000AE9A8FEFA1
:1036C0008ABB8DE685BB1BBAAE980000AE9A8FEF21
:1036D0008ABB80E685BB82E28BBBAE980000AE9AC7
:1036E0001092BE01089580EE85BB8FEF84BB1ABA9D
:1036F00089E00000815087FFFCCFAF9887E893E115
:103700000000019797FFFCCF1ABA88E785BBAD98F8
:10371000000089B3AD9A9FEF9ABB88E785BB9BBB3E
:10372000AE980000AE9A83E60000815087FFFCCF80
:103730000E94AD1A8AB783608ABF89B7806189BF4A
:1037400008958091BE018F5F8093BE018091BE017C
:10375000823310F00E94AD1A089508959C018FEFF6
:103760008ABB80E685BB82E28BBBAE980000AE9A36
:103770008FEF8ABB84E685BB80E48BBBAE980000EC
:10378000AE9A8FEF8ABB88E685BB1BBAAE98000065
:10379000AE9A8FEF8ABB89E685BB80E48BBBAE987F
:1037A0000000AE9A9FEF9ABB87E685BB9BBBAE98A5
:1037B0000000AE9A6C33710588F48FEF8ABB8AE6FD
:1037C00085BB8CE38BBBAE980000AE9A8FEF8ABBB3
:1037D0008BE685BB1BBAAE98000011C08FEF8ABB89
:1037E0008AE685BB6BBBAE980000AE9A8FEF8ABBB2
:1037F0008BE685BB872F99278BBBAE980000AE9ACE
:103800008FEF8ABB80E685BB82E18BBBAE98000060
:10381000AE9A6115710571F04FEF90E7F9019B01C8
:103820004ABB95BB81918BBBAE980000AE9A2150EC
:103830003040B1F79FEF80E72BE330E09ABB85BBC8
:103840001BBAAE980000AE9A2150304037FFF6CF39
:1038500047E621E030E01ABA45BBAD98000089B3D5
:10386000AD9A992756E0969587955A95E1F781701C
:1038700090708217930779F76C33710588F48FEF96
:103880008ABB85E685BB8CE38BBBAE980000AE9A05
:103890008FEF8ABB86E685BB1BBAAE98000011C0CD
:1038A0008FEF8ABB85E685BB6BBBAE980000AE9AF6
:1038B0008FEF8ABB86E685BB872F99278BBBAE9897
:1038C0000000AE9A8FEF8ABB80E685BB84E28BBB9B
:1038D000AE980000AE9A0895FC01DB018FEF8ABB21
:1038E00080E685BB8AE18BBBAE980000AE9A1ABA1F
:1038F00080E785BBAD98000049B3AD9A1ABA85BB85
:10390000AD98000049B3AD9A1ABA85BBAD980000D6
:1039100049B3AD9A1ABA85BBAD98000089B3AD9A88
:103920009927382F2227842F9927282B392B2430A9
:10393000310520F0B9016450704002C060E070E0D1
:103940004D915C9111976417750708F4AB0141150F
:10395000510561F090E79A011ABA95BBAD98000045
:1039600089B38193AD9A21503040B1F74D935C9368
:103970006115710559F080E79B011ABA85BBAD98B6
:10398000000049B3AD9A21503040B9F71ABA87E622
:1039900085BBAD98000049B3AD9A08951F920F9270
:1039A0000FB60F9211240F931F932F933F934F93B2
:1039B0005F936F937F938F939F93AF93BF93EF9397
:1039C000FF93CF93DF93CDB7DEB7C258D240DEBFAF
:1039D000CDBF0E94DC2C8C010E944F1A812F9927A9
:1039E0000E944F1A1ABA87E685BBAD98000089B3CA
:1039F000AD9A80FF37C08E010F571D4F80E892E0CF
:103A0000F80180839183B801CE0101960E946C1C5D
:103A1000A895F80160817181CE0101960E9408127B
:103A20001ABA83E685BBAD98000029B3AD9A8FEF33
:103A30008ABB80E685BB82E68BBBAE980000AE9A5F
:103A40001ABA87E685BBAD98000099B3AD9A8FEF9F
:103A50008ABB80E685BB82E28BBBAE980000AE9A43
:103A6000291749F69FEF9ABB87E685BB9BBBAE98AB
:103A70000000AE9A8FEF8ABB80E685BB82E28BBBEB
:103A8000AE980000AE9A1092BE01CE57DD4FF8946A
:103A9000DEBFCDBFDF91CF91FF91EF91BF91AF918D
:103AA0009F918F917F916F915F914F913F912F9156
:103AB0001F910F910F900FBE0F901F901895282FF8
:103AC00090E0E5E8F5E08081882319F08181821794
:103AD00021F09F5F7A969430B0F39430B0F4892F40
:103AE00099272AE130E0829FF001839FF00D929F99
:103AF000F00D1124EB57FA4F80818150823018F479
:103B000082E0808308951082089590E0E5E8F5E072
:103B100080817A96882319F09F5F9430C8F394309F
:103B200048F48AE1989FF0011124EB57FA4F83E0A3
:103B30008083218308950895282F90E0E5E8F5E03B
:103B40008081882319F08181821721F09F5F7A9606
:103B50009430B0F3943070F48AE1989FF00111240E
:103B6000EB57FA4F80818150823018F482E08083D5
:103B70000895108208950895EF92FF920F931F9376
:103B8000B82FA0E0E5E8F5E08081882319F0818175
:103B90008B1721F0AF5F7A96A430B0F3A43008F011
:103BA00062C08AE1A89FF0011124EB57FA4F80818F
:103BB000A82FBB27A830B10508F055C091E001C07F
:103BC000990FAA95EAF7892F8E7661F594FD03C0C7
:103BD00097FD1EC048C0413151056105710510F5C2
:103BE000C801AA27BB277C018D0180E190E0A0E0FD
:103BF000B0E0841B950BA60BB70B8E159F05A00795
:103C0000B10710F47C018D01E40FF51F3A9624C032
:103C1000403151056105710530F1413251056105B1
:103C2000710518F080E090E020C0C801AA27BB27EA
:103C30007C018D0180E290E0A0E0B0E0841B950B58
:103C4000A60BB70B8E159F05A007B10710F47C01DA
:103C50008D01E40FF51F3697A701BF01C9010E942E
:103C60008530C70102C08FEF9FEF1F910F91FF902A
:103C7000EF900895282F90E0E5E8F5E08081882313
:103C800019F08181821721F09F5F7A969430B0F30A
:103C90009430E8F48AE1989FF0011124EB57FA4F31
:103CA000808199278430910519F0079749F008958C
:103CB000403151056105710550F085E0808308951C
:103CC000403251056105710510F088E08083089548
:103CD0000895AF92BF92CF92DF92EF92FF920F932F
:103CE0001F93CF93DF93A82F5A016B0190E0E5E873
:103CF000F5E08081882319F081818A1721F09F5F88
:103D00007A969430B0F39430B0F58AE1989FE00150
:103D10001124CB57DA4F8881853069F580E1A816E8
:103D2000B104C104D104D0F4FE01EA0DFB1D3A96A2
:103D300040E150E060E070E04A195B096C097D09E0
:103D4000C801AA27BB2784179507A607B70710F451
:103D5000AC01BD01B901CF010E948530C801AA277D
:103D6000BB278A0D9B1DAC1DBD1D4097A105B1054C
:103D700010F086E08883C7018032910510F480E25C
:103D800090E0DF91CF911F910F91FF90EF90DF9026
:103D9000CF90BF90AF900895E5E8F5E083E0108202
:103DA0007A96815087FFFBCF08956F927F928F9212
:103DB0009F92BF92CF92DF92EF92FF920F931F9349
:103DC000CF93DF93CDB7DEB760970FB6F894DEBF21
:103DD0000FBECDBFF89430E04AE150E0209174016D
:103DE0002F5F243008F020E0822F9927849FF00174
:103DF000859FF00D949FF00D1124EB57FA4FE08151
:103E0000E33029F0E63019F03F5F343048F3209377
:103E10007401343010F07894E5C08AE1289F600185
:103E2000112485E895E0C80ED91ED6012C9181E0B9
:103E30008C937894BB24822F99278330910521F0AD
:103E4000069709F43FC0BFC0F89486010E5F1F4F6C
:103E500068E0C8010E94831A7894A5E7B1E0F601F2
:103E600037E08D919281892782873150319637FFD3
:103E7000F8CF38E0E2E1F0E0CE0EDF1ED601F80127
:103E800001900D923A95E1F78EEE9FEFC80ED91E84
:103E900019861A861B861C861D861E861F86188A12
:103EA000C6010A9639E0E32EF12CEC0EFD1E02E06D
:103EB00010E09C01AC0160E487EA91E00E94A52D2E
:103EC00024E07FC0B98629E0822E912C8C0E9D1EA5
:103ED000BA86BB86BC86BD86BE86BF86B88A9AE097
:103EE000692E712C6C0C7D1C740102E010E09301B2
:103EF000A30160E487EA91E00E94D82E3B2DAEE753
:103F0000B1E0F6018D91928189279285981721F46D
:103F10003F5F31963830B0F3383010F428E051C0AC
:103F20009E012F5F3F4F86010E5E1F4F88E0D90133
:103F3000F80101900D928A95E1F789819927009700
:103F400019F0019751F018C0F601128AF8940E94F6
:103F5000451AF8018183789414C0F894F9016281BC
:103F600081810E94071A81E0D8018C930E94451A32
:103F7000F8018183789405C08FEF9FEFD8018D936E
:103F80009C93A7E8B1E0F60137E08D9192818927F3
:103F900082873150319637FFF8CF1986F4011182AC
:103FA000128213821482158216821782740102E033
:103FB00010E09301A30160E487EA91E00E94A52D3F
:103FC00027E081E0B82EF894D6018C91823011F46C
:103FD0001C9207C0F6012083BB2019F081810E944A
:103FE000332C789460960FB6F894DEBF0FBECDBF29
:103FF000DF91CF911F910F91FF90EF90DF90CF90C5
:10400000BF909F908F907F906F900895E5EFF5E0BF
:1040100087E01082F096815087FFFBCF08950F93C1
:104020001F93CF93DF93EC018B01842F422F282F16
:104030003327C901C6966817790708F441C0295E7D
:104040003F4F2C733070322F2227330F330F842FC2
:1040500099278F739070282B392B832F9927322F14
:104060002227822B932B8EA79FA71AAA1BAA1CAAD2
:104070001DAA80910C018A8F80910D018B8F8091F8
:104080000E018C8F80910F018D8FC8018297B8012E
:104090006A5170409C0146E050E0CE014A960E9471
:1040A000200C9C01892F9927322F2227822B932BBA
:1040B0008AAB9BAB86E08F8BB801CE010E94F516D0
:1040C000DF91CF911F910F9108956F927F928F9200
:1040D0009F92AF92BF92CF92DF92EF920F931F9376
:1040E000CF93DF93CDB7DEB7E6970FB6F894DEBF78
:1040F0000FBECDBFFC015A016B013801490124817B
:104100003581832F9927322F2227822B932B8BA344
:104110009CA326813781832F9927322F2227822B38
:10412000932B8DA39EA38D2D9927AA27BB27A6018C
:104130009501207030705070232F342F452F552754
:10414000822B932BA42BB52BA601950120704070D8
:104150005070542F432F322F2227822B932BA42BC6
:10416000B52B5A2D442733272227822B932BA42BA0
:10417000B52B8FA398A7A9A7BAA7892D9927AA27F6
:10418000BB27A4019301207030705070232F342F6F
:10419000452F5527822B932BA42BB52BA4019301DC
:1041A000207040705070542F432F322F2227822BC3
:1041B000932BA42BB52B562D442733272227822B54
:1041C000932BA42BB52B8BA79CA7ADA7BEA723A190
:1041D00034A1832F9927322F2227822B932B89AB4F
:1041E0009AAB80818F8F818188A3828189A383810B
:1041F0008AA32E2D40E066E370E0CE0101960E9476
:104200000F20E6960FB6F894DEBF0FBECDBFDF914C
:10421000CF911F910F91EF90DF90CF90BF90AF9013
:104220009F908F907F906F9008956F927F928F9262
:104230009F92AF92BF92CF92DF92EF920F931F9314
:10424000CF93DF93CDB7DEB7EA970FB6F894DEBF12
:104250000FBECDBFFC015A016B0138014901248119
:104260003581832F9927322F2227822B932B8BA3E3
:104270009CA326813781832F9927322F2227822BD7
:10428000932B8DA39EA38D2D9927AA27BB27A6012B
:104290009501207030705070232F342F452F5527F3
:1042A000822B932BA42BB52BA60195012070407077
:1042B0005070542F432F322F2227822B932BA42B65
:1042C000B52B5A2D442733272227822B932BA42B3F
:1042D000B52B8FA398A7A9A7BAA7892D9927AA2795
:1042E000BB27A4019301207030705070232F342F0E
:1042F000452F5527822B932BA42BB52BA40193017B
:10430000207040705070542F432F322F2227822B61
:10431000932BA42BB52B562D442733272227822BF2
:10432000932BA42BB52B8BA79CA7ADA7BEA723A12E
:1043300034A1832F9927322F2227822B932B89ABED
:104340009AAB80818F8F818188A3828189A38381A9
:104350008AA382E08FAB34E038AF81E090E089AF90
:104360009AAF2E2D432F6AE370E0CE0101960E9492
:104370000F20EA960FB6F894DEBF0FBECDBFDF91D7
:10438000CF911F910F91EF90DF90CF90BF90AF90A2
:104390009F908F907F906F9008958F929F92AF9291
:1043A000BF92CF92DF92EF92FF920F931F93CF9322
:1043B000DF93CDB7DEB7C653D1400FB6F894DEBF5A
:1043C0000FBECDBFF82E6B01E42EFB01808584303B
:1043D00019F0873009F072C0F601818992898C0149
:1043E0002227332745855685678570898185928583
:1043F000A385B4854A015B01881A990AAA0ABB0AF7
:10440000081919092A093B0981A592A5AA27BB27E2
:10441000081719072A073B0710F4D901C8015C01E6
:1044200021E08130920720F0A12C21E0B22E03C0C0
:10443000892B09F446C0F60126A537A5838D948DF6
:10444000A58DB68D481B590B6A0B7B0B4150504014
:1044500060407040F901A481B58185019E01295C0D
:104460003F4F8F2DFD010995A816B90628F591E15A
:10447000E92EF601078D10A121A132A145855685AF
:1044800067857089C6010E946520F601858596853D
:10449000A785B0890196A11DB11D85879687A7873D
:1044A000B08B85E08087A6A5B7A5FD012281338169
:1044B0008F2DF9010995ACC05C0103C0AA24BB246F
:1044C00003C0A114B10419F4EE2009F4A1C0F6014F
:1044D00024813581832F9927322F2227822B932BFA
:1044E0008BA39CA326813781832F9927322F2227E4
:1044F000822B932B8DA39EA3E584F68407851089D8
:10450000812F9927AA27BB27A80197012070307017
:104510005070232F342F452F5527822B932BA42BFC
:10452000B52BA8019701207040705070542F432F75
:10453000322F2227822B932BA42BB52B5E2D4427C1
:1045400033272227822B932BA42BB52B8FA398A73D
:10455000A9A7BAA7E78CF0A001A112A1812F9927E2
:10456000AA27BB27A8019701207030705070232F15
:10457000342F452F5527822B932BA42BB52BA80125
:104580009701207040705070542F432F322F2227F4
:10459000822B932BA42BB52B5E2D44273327222768
:1045A000822B932BA42BB52B8BA79CA7ADA7BEA7C3
:1045B00023A134A1832F9927322F2227822B932BDB
:1045C00089AB9AAB80818F8F818188A3828189A3F7
:1045D00083818AA3A114B10411F028E101C020E174
:1045E000C501C69640E0BC01CE0101960E940F2095
:1045F000950144275527F60185859685A785B089BD
:10460000820F931FA41FB51F85879687A787B08B3E
:10461000CA5CDE4F0FB6F894DEBF0FBECDBFDF9190
:10462000CF911F910F91FF90EF90DF90CF90BF90AF
:10463000AF909F908F9008958F929F92AF92BF926C
:10464000CF92DF92EF92FF920F931F93CF93DF935E
:10465000FF24CDEED5E0CC24DD249885992309F400
:1046600075C08BA58F5F8BA79A3011F495E001C0C0
:1046700094E18BA5891708F469C01BA68885992742
:104680008530910509F448C0863091054CF483309B
:10469000910599F0843091052CF50297A9F056C048
:1046A0008A30910534F488309105B4F50797D1F03C
:1046B0004DC00A9709F449C049C0E2E1EE2E0F8DC2
:1046C00018A129A13AA106C072E0E72E00E010E08F
:1046D00020E030E049855A856B857C85CE010E94BB
:1046E000152127C029853A854B855C858D859E855A
:1046F000AF85B88949015A01881A990AAA0ABB0AE2
:10470000B7FE04C02D873E874F87588B40E0BE011F
:104710008F2D0E94CD211AC061E1E62E0F8D18A1C8
:1047200029A13AA149855A856B857C85CE010E94D5
:10473000652089859A85AB85BC850196A11DB11D33
:104740008D879E87AF87B88B01C0188688858823A0
:10475000A1F18CA58F5F8CA7823378F154E0E52E10
:104760000F8D18A129A13AA149855A856B857C85B1
:10477000CE010E9465208885282F332728303105F7
:1047800080F481E001C0880F2A95EAF7887949F022
:104790001886EEA5FFA50280F381E02D8F2D0995E7
:1047A0000CC080E390E0C89EF001C99EF00DD89E39
:1047B000F00D1124E351FA4F108688858823A1F16A
:1047C0008DA58F5F8DA7863978F144E0E42E0F8D9B
:1047D00018A129A13AA149855A856B857C85CE010E
:1047E0000E9465208885282F33272830310580F4E2
:1047F00081E001C0880F2A95EAF7887949F0188688
:10480000EEA5FFA50280F381E02D8F2D09950CC048
:1048100080E390E0C89EF001C99EF00DD89EF00D97
:104820001124E351FA4F1086F3940894C11CD11C53
:10483000E09637E0932E9F1408F00FCFDF91CF91D1
:104840001F910F91FF90EF90DF90CF90BF90AF90AE
:104850009F908F9008952F923F924F925F926F9208
:104860007F928F929F92AF92BF92CF92DF92EF9200
:10487000FF920F931F93CF93DF93CDB7DEB7CB5447
:10488000D0400FB6F894DEBF0FBECDBF8FAB98AF50
:104890008B016633710508F49DC66EEDC62E6FEF71
:1048A000D62EC00ED11EC8014A97960146E050E0B0
:1048B000BC018FA998AD4A960E94200C892B09F063
:1048C00089C6EFA9F8AD84A195A1692F7727982F04
:1048D0008827682B792B82A193A1E92EFF24982F9A
:1048E0008827E82AF92A6115710509F473C6E114CD
:1048F000F10409F46FC626A137A140A551A5852E64
:104900009924AA24BB24DA01C90180709070B07088
:10491000892F9A2FAB2FBB27882A992AAA2ABB2A2C
:10492000DA01C9018070A070B070BA2FA92F982F3A
:104930008827882A992AAA2ABB2AB22FAA27992728
:104940008827882A992AAA2ABB2A22A533A544A502
:1049500055A5452E552466247724DA01C9018070B7
:104960009070B070892F9A2FAB2FBB27482A592AF5
:104970006A2A7B2ADA01C9018070A070B070BA2F50
:10498000A92F982F8827482A592A6A2A7B2AB22FCA
:10499000AA2799278827482A592A6A2A7B2A80A980
:1049A00091A9292F3327982F8827282B392B2DAF12
:1049B0003EAF48E152E021964EAF5FAF219726A56A
:1049C00037A5832F99278F7327968FAF2797369513
:1049D0002795369527952C73307023962EAF3FAFD1
:1049E00023972431310508F4F5C5C216D30608F41F
:1049F000F1C5021B130B0252104025960EAF1FAFDC
:104A0000259722962FAD22972451F6962223A1F1C5
:104A1000808199278130910549F0823091051CF4FD
:104A2000892B51F11CC0029721F019C021503196F9
:104A3000EDCF243008F4CEC58181843009F0CAC599
:104A400082819381A92FBB27982F8827A82BB92B68
:104A50002196AEAFBFAF219724503496D7CF2230E6
:104A600018F08181281718F4E0E0F0E020E081815F
:104A7000281BE80FF11DCACFEF2B09F4ABC5259613
:104A80000EAD1FAD2597222733272B960CAF1DAFF8
:104A90002EAF3FAF2B97080D191D2A1D3B1D09AFE7
:104AA0001AAF2BAF3CAF27961FAD2797212E33248B
:104AB00021FE0CC029AD3AAD4BAD5CAD2F5F3F4F31
:104AC0004F4F5F4F29AF3AAF4BAF5CAF20FE0BC0EB
:104AD00089AD9AADABADBCAD0196A11DB11D89AF3D
:104AE0009AAFABAFBCAF26961FAE2697ADEEB5E042
:104AF000FD018085882331F19C91EFA9F8AD828D6D
:104B0000981701F5FD019181EFA9F8AD838D9817F4
:104B1000C9F4FD019281EFA9F8AD848D981791F445
:104B2000FD019381EFA9F8AD858D981759F4FD012A
:104B3000848195818617970729F4868197818E1540
:104B40009F0551F02696FFAD2697FF5F2696FFAF93
:104B50002697D096F83060F226960FAD269708304B
:104B600008F46BC027961FAD2797123009F065C077
:104B700025962EAD3FAD2597232B09F05EC0809181
:104B80000201909103016817790729F4A0E2B0E0CF
:104B90004AE651E00CC08091000190910101681734
:104BA000790709F04AC0A0E0B1E046E151E026965D
:104BB0001FAE2697E5EFF5E08081F096882349F057
:104BC00026963FAD26973F5F26963FAF2697383013
:104BD00098F326968FAD2697883078F5282F3327BF
:104BE00080E390E0289FF001299FF00D389FF00DA1
:104BF00011249F0123513A4FEFA9F8AD828DF9019D
:104C00008083EFA9F8AD838DF9018183EFA9F8AD19
:104C1000848DF9018283EFA9F8AD858DF901838335
:104C200064837583E682F78281E0808713A614A6E9
:104C300015A6A3A3B4A346A757A72696FFAD26970C
:104C4000F83008F493C0C10196958795969587959D
:104C5000AC014170507080FDBDC4872F9927362F5D
:104C60002227822B932B8BA39CA38F2D99273E2D3C
:104C70002227822B932B8DA39EA349AB5AABEFA97E
:104C8000F8AD828D8F8F838D88A3848D89A3858DC8
:104C90008AA324FE30C0872D9927AA27BB27A3010A
:104CA0009201207030705070232F342F452F5527DC
:104CB000822B932BA42BB52BA30192012070407063
:104CC0005070542F432F322F2227822B932BA42B4B
:104CD000B52B542D442733272227822B932BA42B2B
:104CE000B52B8FA398A7A9A7BAA71BA61CA61DA67C
:104CF0001EA624E033C01FA218A619A61AA6E9AC66
:104D0000FAAC0BAD1CAD812F9927AA27BB27A801B0
:104D10009701207030705070232F342F452F552766
:104D2000822B932BA42BB52BA801970120704070E8
:104D30005070542F432F322F2227822B932BA42BDA
:104D4000B52B5E2D442733272227822B932BA42BB0
:104D5000B52B8BA79CA7ADA7BEA724E140E066E3D7
:104D600070E0CE0101960E940F2034C480E32696A5
:104D70000FAD2697089F600111242DEE35E0C20E7D
:104D8000D31E25FE0DC024FC74C284E1E82E09ADBB
:104D90001AAD2BAD3CAD40E050E060E070E098C251
:104DA000F601F0852C96FFAF2C978F2F9927813035
:104DB000910521F0029709F45EC001C122FC0AC4EA
:104DC00024FE09C004E0E02E00E010E020E030E026
:104DD000B301A201E1C021FEFDC30894811C911C16
:104DE000A11CB11CF601878E90A2A1A2B2A20894C8
:104DF00081089108A108B10885A296A2A7A2B0A631
:104E000064E0C6014B960E94831A12E1E12EF6017E
:104E1000078D10A121A132A1438D548D658D768D12
:104E2000C6010E941521F601838D948DA58DB68D46
:104E30000196A11DB11D85879687A787B08B019725
:104E4000A109B10981879287A387B48783E080870E
:104E5000EDACFEACE18AF28A838A948AA58AB68A8E
:104E6000478A508E618E728E2196EEACFFAC2197F0
:104E7000E1A6F2A6A2C060E024FE31C0F601838D57
:104E8000948DA58DB68D83017201E81AF90A0A0B7B
:104E90001B0B1E141F04100611067CF485859685D5
:104EA000A785B08993018201081B190B2A0B3B0BC4
:104EB00010161106120613061CF422FC8BC3D9C16E
:104EC000F60181859285A385B48584199509A60983
:104ED000B709181619061A061B060CF061E022FE27
:104EE00004C0662309F476C380C1662311F424FC50
:104EF00071C321FE6FC3D501C4010196A11DB11D6F
:104F0000F601878F90A3A1A3B2A385A296A2A7A220
:104F1000B0A6878B908FA18FB28F662321F0418638
:104F2000528663867486EDACFEACF601E18AF28AA5
:104F3000838A948AA58AB68A478A508E618E728E39
:104F40002196EEACFFAC2197E1A6F2A68185928571
:104F5000A385B485438D548D658D768D841B950B0B
:104F6000A60BB70B181619061A061B06CCF484E01C
:104F70008087A6A5B7A5ED91FC9126968FAD2697C3
:104F80000995B0E1EB2EF601078D10A121A132A108
:104F90004585568567857089C6010E9465200CC0CD
:104FA00083E0F6018087A2E1EA2E078D10A121A1FE
:104FB00032A1C6010E941521F60113A60BC3F6010A
:104FC00063A174A12596EEACFFAC2597EF2851F5AF
:104FD000278D30A141A152A16115710539F48216C6
:104FE0009306A406B50609F0F5C266C0DA01C90148
:104FF00088199909AA09BB09181619061A061B0669
:105000000CF4E8C2CB01AA27BB27280F391F4A1F7F
:105010005B1FD501C401821B930BA40BB50BB7FF1B
:10502000D9C24AC06115710509F4D4C2F601E78CF2
:10503000F0A001A112A1D801C70188199909AA09F4
:10504000BB09181619061A061B067CF0CB01AA2705
:10505000BB278E0D9F1DA01FB11FA5019401281B0A
:10506000390B4A0B5B0B57FD27C02B962CAD3DAD82
:105070004EAD5FAD2B97280D391D4A1D5B1DD80124
:10508000C701821B930BA40BB50B8F5F9F4FAF4FD4
:10509000BF4F09F09FC2CB01AA27BB27E80EF91E1C
:1050A0000A1F1B1F2E193F09400B510B2150304086
:1050B000404050400AF08EC261E0F601278D30A1D9
:1050C00041A152A1D501C401821B930BA40BB50BC6
:1050D000181619061A061B060CF47CC2662309F47E
:1050E00079C2878D90A18819990901F121FE08C024
:1050F0002796FFAD2797FD7F2796FFAF279701974C
:105100002396EEACFFAC2397E80EF91E2396EEAE85
:10511000FFAE239725960EAD1FAD2597081B190BE3
:1051200025960EAF1FAF259749015A01F60123A11D
:1051300034A12596EEACFFAC25972E153F05A8F4BB
:10514000E21AF30AC701AA27BB2749AD5AAD6BADD6
:105150007CAD481B590B6A0B7B0B49AF5AAF6BAF49
:105160007CAF25962EAF3FAF2597F60113A6279665
:10517000FFAD27972F2E332422FE10C02C96EFACC4
:105180002C978E2D99278830910534F48430910521
:10519000F4F40397E1F002C00B973CF121FE27C025
:1051A000F60180859927833091050CF188309105AF
:1051B0001CF00B97E4F40EC034E0E32E00E010E0A6
:1051C00020E030E0B301A201C6010E946520F60193
:1051D0001086CFC124E0E22E00E010E020E030E0B5
:1051E000B301A201C6010E946520F6011AC124FE86
:1051F000F1C1F60180859927883091053CF484300F
:1052000091050CF03FC0039761F018C189309105FA
:10521000C9F1893091050CF4F6C00A9709F403C16D
:105220000DC1F60181859285A385B4858419950900
:10523000A609B709181619061A061B06D4F08585A3
:105240009685A785B08983017201E81AF90A0A0BCD
:105250001B0B1E141F04100611065CF084E08087EF
:10526000A6A5B7A5ED91FC9126968FAD2697099539
:1052700009C094E0E92E00E010E020E030E0B30146
:10528000A20126C0F60181859285A385B48583019C
:105290007201E81AF90A0A0B1B0B1E141F041006F0
:1052A00011060CF0CBC04585568567857089D30102
:1052B000C201841B950BA60BB70B181619061A060C
:1052C0001B0654F480E1E82E078D10A121A132A124
:1052D000C6010E9465207EC1F60141865286638622
:1052E00074862389348945895689DA01C901881968
:1052F0009909AA09BB09B7FD12C0281539054A0545
:105300005B05D1F48789908DA18DB28D84199509A3
:10531000A609B709181619061A061B066CF0EDAC9B
:10532000FEACF601E18AF28A838A948AA58AB68A5B
:10533000478A508E618E728EF60114A666A577A5F7
:1053400081859285A385B485238D348D458D568DB9
:10535000821B930BA40BB50B0197A109B109FB01AB
:1053600026813781AC01BD0126968FAD2697F901C4
:105370000995F6018085992786309105C9F0873017
:1053800091051CF4059721F059C0099751F156C0B9
:10539000F601218532854385548585859685A785C7
:1053A000B089281739074A075B0711F486E0808720
:1053B000F601218532854385548585859685A785A7
:1053C000B089281739074A075B07C1F5A6A5B7A515
:1053D000FD012281338126968FAD2697F90109952B
:1053E0002DC0F601218532854385548585859685B6
:1053F000A785B089281739074A075B0709F0EAC073
:105400008AE080871BC0F60121853285438554855B
:1054100085859685A785B089281739074A075B07D0
:1054200069F41086D7C000E1E02E09AD1AAD2BADAE
:105430003CADB301A201C6010E94652040E0259663
:10544000EEACFFAC2597E114F10409F453C0F6016A
:10545000808599270497039708F04CC063A174A135
:105460006E197F0963A374A325962EAD3FAD2597D2
:10547000790100271127878D90A1A1A1B2A18E0DDE
:105480009F1DA01FB11F878F90A3A1A3B2A344A704
:10549000A6A4B7A42FA938AD23964EAD5FAD239730
:1054A000240F351F2E5D3F4F2FAB38AF25A136A1FE
:1054B00047A150A5821B930BA40BB50B8E199F0916
:1054C000A00BB10B0197A109B109F501A084B1842A
:1054D0007B0125960EAD1FAD25972FA938ADAC01E8
:1054E000BD0126968FAD2697F5010995F60183A398
:1054F00094A341E020FE68C0F6018085992785309D
:10550000910509F441C08630910524F403970CF409
:105510005BC008C08630910509F445C00B970CF0BC
:1055200053C051C0F601878D90A1A1A1B2A10196EF
:10553000A11DB11D878F90A3A1A3B2A327E020874F
:1055400011E1E12E8C019D014585568567857089A5
:10555000C6010E946520F60185859685A785B089DC
:105560000196A11DB11D85879687A787B08B89E01D
:105570008087A6A5B7A5FD012281338126968FAD30
:105580002697F901099526C041E0F601878D90A183
:10559000A1A1B2A10196A11DB11D878F90A3A1A3C6
:1055A000B2A389E00EC041E0F601878D90A1A1A1D0
:1055B000B2A10196A11DB11D878F90A3A1A3B2A393
:1055C0008AE0808701C041E0B60126968FAD26971C
:1055D0000E94CD21C55BDF4F0FB6F894DEBF0FBE32
:1055E000CDBFDF91CF911F910F91FF90EF90DF9092
:1055F000CF90BF90AF909F908F907F906F905F9073
:105600004F903F902F9008956F927F928F929F922C
:10561000AF92BF92CF92DF92EF920F931F93CF93EF
:10562000DF93DC01EA01390120919A0130919B015D
:1056300040E0EDEEF5E08085882329F084819581B6
:105640008217930721F04F5FF0964830A0F3C9010D
:105650000196483010F49C01EBCF90939B0180930E
:105660009A018050904C30F080E090E890939B013C
:1056700080939A0140E0E5EFF5E08081F096882381
:1056800019F04F5F4830C8F3483018F08FEF90E0C2
:1056900067C0842E992480E390E0889E6001899EF3
:1056A000D00C989ED00C11248DEE95E0C80ED91E1A
:1056B0008C91F6018083FD018181F6018183FD01DA
:1056C0008281F6018283FD018381F6018383248335
:1056D000358366837783178E10A211A212A215A2BA
:1056E00016A217A210A680E3489F5001112464E07F
:1056F000C501885F994F0E94831A72E0E72E00E08F
:1057000010E020E030E0F601438D548D658D768DFC
:10571000C50183519A4F0E941521F601838D948D06
:10572000A58DB68D81879287A387B4870196A11D29
:10573000B11D85879687A787B08BE086118A128A6C
:10574000138A148A158A168A178A108E118E128E61
:1057500013A614A615A6C3A3D4A366A677A6C40150
:10576000DF91CF911F910F91EF90DF90CF90BF907D
:10577000AF909F908F907F906F900895EF92FF92DF
:105780000F931F93CF93DF93F82E87E08F1508F4C4
:1057900063C02F2D332780E390E0289FF001299FDD
:1057A000F00D389FF00D1124E351FA4F80858823C6
:1057B00009F452C080E3F89EE0011124C351DA4F8E
:1057C00088859927853091053CF4833091054CF408
:1057D00001970CF441C003C00797E9F03DC018865B
:1057E0003BC0F1E1EF2E0F8D18A129A13AA14D8503
:1057F0005E856F857889CE010E9465208D859E85A6
:10580000AF85B8890196A11DB11D8D879E87AF8791
:10581000B88B85E019C0E1E1EE2E0F8D18A129A10A
:105820003AA14D855E856F857889CE010E946520FD
:105830008D859E85AF85B8890196A11DB11D8D8787
:105840009E87AF87B88B89E08887EEA5FFA5028089
:10585000F381E02D8F2D0995DF91CF911F910F914D
:10586000FF90EF900895CF93C82F883078F5282FB8
:10587000332780E390E0289FF001299FF00D389FA7
:10588000F00D1124E351FA4F80858823F9F080E36D
:10589000C89FF0011124E351FA4F80859927843085
:1058A000910511F0079791F4218532854385548540
:1058B00085859685A785B089281739074A075B072C
:1058C00029F440E0BF018C2F0E94CD21CF91089593
:1058D0000895089580E090E008950895EF92FF9272
:1058E000C7018038910510F480E890E0FF90EF90B8
:1058F00008951F920F920FB60F9211242F933F938A
:105900004F935F936F937F938F939F93AF93BF93C7
:10591000EF93FF930E9469188091C0018F5F80937D
:10592000C0018091BF018F5F8093BF018091BF0153
:10593000843610F01092BF018091BF019927823305
:105940009105B1F08333910534F48A30910551F01B
:105950004E9759F015C08634910569F08A35910546
:1059600069F00EC00E94040A0BC00E94CD1508C049
:105970000E94A11B05C00E941C2302C00E94F12CA2
:10598000FF91EF91BF91AF919F918F917F916F9117
:105990005F914F913F912F910F900FBE0F901F90ED
:1059A00018958EE083BF8CE781BF87B7826087BF81
:1059B0001FBC81E08EBD08958CB59DB5089588E02B
:1059C0008AB987E689B940E050E0BA018BEE9CE2E3
:1059D0000E942F3008955D9BFECF8CB980E090E04F
:1059E00008958091C2018F5F8093C2018A3048F090
:1059F0001092C2018091C101833018F48F5F8093AF
:105A0000C101089508950F931F93CF93DF93EC0185
:105A10008B016A327105B8F1CB018297292F3327A8
:105A2000982F8827282B392B2EA33FA318A619A619
:105A300080910C018A8F80910D018B8F80910E01D6
:105A40008C8F80910F018D8F832F9927322F2227E2
:105A5000822B932BB8016A5170409C0141E150E0C8
:105A6000CE014A960E94200C9C01892F9927322F43
:105A70002227822B932B88A799A781E18F8BB801CE
:105A8000CE010E94F516DF91CF911F910F910895DD
:105A90000F931F93CF93DF93EC019B016A32710543
:105AA00008F44EC08AA19BA1892B09F449C08CA19E
:105AB0009DA1892B09F444C08EA19FA1692F77274E
:105AC000982F8827682B792B8B010E5D1F4F20178D
:105AD0003107B0F19B0141E150E0685F7F4FCE019B
:105AE0004A960E94200C892B59F58CA19DA1292F43
:105AF0003327982F8827282B392B2730310501F59C
:105B00008AA19BA180509740D9F08091C101882340
:105B1000B9F081508093C1018AA19BA18CA39DA360
:105B200080E097E08AA39BA38A8D8E8F8B8D8F8FC9
:105B30008C8D88A38D8D89A3B801CE010E94032D81
:105B4000DF91CF911F910F9108952F923F924F9225
:105B50005F926F927F928F929F92AF92BF92CF92FD
:105B6000DF92EF92FF920F931F93CF93DF93CDB706
:105B7000DEB76B970FB6F894DEBF0FBECDBF898B33
:105B80009A8B6B8BEC8AFD8A0115110509F4F7C01D
:105B9000288F398F4A8F5B8F0E8B1F8BAA8DBB8D01
:105BA0002C90FD0131804280538064807580868016
:105BB0009780AC89BD89AC90FD01B180C280D38053
:105BC000E480F58006811781222D2A25332D3B257F
:105BD000442D4C25552D5D25662D6E25772D7F2571
:105BE000882D8027992D912729833A834B835C83C5
:105BF0006D837E838F8398876B89E980FA800B8120
:105C00001C81AD80BE80CF80D88466247724430178
:105C1000662309F47DC0A6019501E4E0220F331F3D
:105C2000441F551FEA95D1F7D601C50175E0B69519
:105C3000A795979587957A95D1F7282739274A27E9
:105C40005B272A0D3B1D4C1D5D1DF301E370F070B9
:105C5000EE0FFF1FEE0FFF1F89899A89E80FF91FCA
:105C600080819181A281B381860D971DA81DB91DE8
:105C7000282739274A275B27E20EF31E041F151F2A
:105C800089EB99E7A7E3BEE9680E791E8A1E9B1E81
:105C9000A8019701F4E0220F331F441F551FFA9506
:105CA000D1F7D801C701E5E0B695A79597958795F7
:105CB000EA95D1F7282739274A275B272E0D3F1D64
:105CC000401F511FD401C3017BE0B695A79597955E
:105CD00087957A95D1F7FC01E370F070EE0FFF1F06
:105CE000EE0FFF1FA989BA89EA0FFB1F80819181FE
:105CF000A281B381860D971DA81DB91D28273927BC
:105D00004A275B27A20EB31EC41ED51E615080CF4A
:105D1000E986FA860B871C87AD86BE86CF86D88A31
:105D20007985E88DF98D70836A8561835B855283FF
:105D30004C8543833D8534832E8525839F859683BB
:105D400088898783AC89BD897C93FD0161835283F7
:105D5000438334832583968387838E899F89019724
:105D60008E8B9F8BAA8DBB8D1896AA8FBB8FE88DCB
:105D7000F98D3896E88FF98F892B09F00FCF6B9644
:105D80000FB6F894DEBF0FBECDBFDF91CF911F914C
:105D90000F91FF90EF90DF90CF90BF90AF909F90CA
:105DA0008F907F906F905F904F903F902F900895CD
:105DB0002F923F924F925F926F927F928F929F921B
:105DC000AF92BF92CF92DF92EF92FF920F931F9309
:105DD000CF93DF93CDB7DEB7A4970FB6F894DEBFAD
:105DE0000FBECDBF898B9A8B6B8BCA01B901EC8A30
:105DF000FD8A0115110509F419C129EB39E747E3BB
:105E00005EE969A37AA38BA39CA30E8B1F8BABA126
:105E1000BCA18C918983FD0181818A8382818B83DE
:105E200083818C8384818D8385818E8386818F831A
:105E300087818887FB89F88F69807A808B809C8036
:105E40002D803E804F8058848F2F9927AA27BB270B
:105E5000BC01CD010E94A8325B016C01688D6623F4
:105E600009F481C084017301E4E0EE0CFF1C001F03
:105E7000111FEA95D1F7D401C30175E0B695A79536
:105E8000979587957A95D1F7E826F9260A271B2753
:105E9000E60CF71C081D191DD601C5016BE0B6956F
:105EA000A795979587956A95D1F7FC01E370F070F7
:105EB000EE0FFF1FEE0FFF1F89899A89E80FF91F68
:105EC00080819181A281B3818A0D9B1DAC1DBD1D76
:105ED000E826F9260A271B272E183F08400A510AF0
:105EE00087E496E8A8ECB1E6A80EB91ECA1EDB1E30
:105EF0008201710174E0EE0CFF1C001F111F7A95E6
:105F0000D1F7D201C10165E0B695A7959795879520
:105F10006A95D1F7E826F9260A271B27E20CF31C1D
:105F2000041D151DF501E370F070EE0FFF1FEE0F5D
:105F3000FF1FA989BA89EA0FFB1F80819181A28185
:105F4000B3818A0D9B1DAC1DBD1DE826F9260A27CD
:105F50001B276E187F08800A910AB88DB150B88F40
:105F6000BB2309F07FCF69867A868B869C862D8637
:105F70003E864F86588AE985E98FFA85FA8F6B85C8
:105F80006B8F8C858C8F9D859D8FAE85AE8FBF85E9
:105F9000BF8FE889E8A3AC89BD892C90FD013180D1
:105FA000428053806480758086809780A98CA2246B
:105FB000BA8CB324C62EC424D82ED524E92EE624C8
:105FC000FE8CF7240F8D082518A11925A9A1BAA1C7
:105FD000AC92FD01B182C282D382E482F582068353
:105FE00017838981AC89BD898C938A81FD01818366
:105FF0008B8182838C8183838D8184838E81858351
:106000008F818683888587838E899F8901978E8B70
:106010009F8BABA1BCA11896ABA3BCA3E9A1FAA12D
:106020003896E9A3FAA3892B09F0F1CEA4960FB60E
:10603000F894DEBF0FBECDBFDF91CF911F910F91BE
:10604000FF90EF90DF90CF90BF90AF909F908F9098
:106050007F906F905F904F903F902F9008950F9397
:106060001F93CF93DF938C01EB010097A1F16CE0BC
:1060700070E081E090E00E947431FC01892B21F1F5
:10608000209751F0C287D38721E0238380916D0749
:1060900090916E07892BD1F001151105A9F00087A9
:1060A0001187038102600383A0916F07B09170078D
:1060B000AB2B51F4F0937007E0936F07C091710719
:1060C000D0917207CD2B51F0CF010DC0F0936E0728
:1060D000E0936D07E1CF672B51F605C0F09372078F
:1060E000E0937107F1CFDF91CF911F910F91089548
:1060F000FB01DC0104C08D910190801921F4415015
:106100005040C8F7881B990B0895FB01DC0102C0C1
:1061100001900D9241505040D8F70895AF92BF9230
:10612000CF92DF92EF92FF920F931F93CF93DF9363
:10613000EC01E880F9800A811B81C801B7012DE1DB
:1061400033EF41E050E00E94C73259016A01C801B3
:10615000B7012DE133EF41E050E00E94C732DC018E
:10616000CB01BC01CD0127EA31E440E050E00E94C0
:10617000A8327B018C01C601B50124E13BE040E07F
:1061800050E00E94A832DC01CB01E81AF90A0A0BA0
:106190001B0B1E141F041006110644F02FEF3FEFD7
:1061A0004FEF5FE7E20EF31E041F151FE882F9822E
:1061B0000A831B834FEF5FEF6FEF7FE7E422F52247
:1061C00006231723C801B701DF91CF911F910F91CB
:1061D000FF90EF90DF90CF90BF90AF900895AF9277
:1061E000BF92CF92DF92EF92FF920F931F93E090B6
:1061F0009C01F0909D0100919E0110919F01C801AA
:10620000B7012DE133EF41E050E00E94C732590160
:106210006A01C801B7012DE133EF41E050E00E946F
:10622000C732DC01CB01BC01CD0127EA31E440E0FB
:1062300050E00E94A8327B018C01C601B50124E127
:106240003BE040E050E00E94A832DC01CB01E81ABC
:10625000F90A0A0B1B0B1E141F041006110644F04A
:106260002FEF3FEF4FEF5FE7E20EF31E041F151F06
:10627000E0929C01F0929D0100939E0110939F017A
:106280004FEF5FEF6FEF7FE7E422F522062317233E
:10629000C801B7011F910F91FF90EF90DF90CF9051
:1062A000BF90AF900895DC01CB0180939C01909347
:1062B0009D01A0939E01B0939F010895FB01DC0115
:1062C0004150504070F08D913191232F2062213642
:1062D00024F02B3714F430628062831B19F43323CB
:1062E00079F7881B990B08950F931F93CF93DF9332
:1062F000869F8001879F100D969F100D1124C80165
:106300000E949031EC01009729F0A80160E070E054
:106310000E94A132CE01DF91CF911F910F9108957C
:10632000CF93DF939C01029710F422E030E040E02D
:1063300050E06091750770917607FB01DA016115F5
:10634000710569F1808191818217930709F452C028
:106350002817390738F44115510519F084179507A6
:1063600008F4AC01DF010280F381E02D309751F792
:1063700041155105A1F0DA01A21BB30B149708F4E3
:1063800043C0DB010AC06D917C91119764177507BA
:1063900009F450C0FD01A281B3811097A1F7E091EB
:1063A0007307F0917407309741F4E091A201F091E6
:1063B000A301F0937407E09373074091A0015091FB
:1063C000A1014115510529F14E1B5F0B42175307DF
:1063D000E8F0C901029648175907C0F0EF01C20F53
:1063E000D31F2296D0937407C093730721933193E0
:1063F000CF0142C01097B1F082819381ED018A8371
:106400009B83CF01029638C09A01BBCF80E090E019
:1064100033C04DB75EB7A091A401B091A5014A1B4E
:106420005B0BD2CF2281338130937607209375079F
:10643000CF01E8CF2417350761F0EA01C21BD30B67
:10644000FD01EC0FFD1F219331932297CD93DC9337
:10645000CFCF309741F0ED014A815B814283538376
:10646000CD01029609C0FD01828193819093760748
:1064700080937507CD01F5CFDF91CF910895CF932C
:10648000DF93009709F45AC0DC011297ED011A82DC
:106490001B8280917507909176070097D9F1FC01D6
:1064A00040E050E0EA17FB0748F4AF010280F381B7
:1064B000E02D3097A1F0EA17FB07B8F3ED01EA836E
:1064C000FB832D913C911197E901CA0FDB1FCE018F
:1064D00002968E179F0719F141155105D9F0EA016F
:1064E000AA83BB83CA01029628813981820F931F38
:1064F0008A179B0719F56D917C911197260F371F0D
:106500002E5F3F4F28833983FD01428153814A83A7
:106510005B8314C0B0937607A09375070FC06A81A0
:106520007B81260F371F2E5F3F4F2D933C93119792
:1065300022813381FD0122833383CECFDF91CF913E
:106540000895DC0101C06D9341505040E0F708957B
:10655000629FD001739FF001829FE00DF11D649F47
:10656000E00DF11D929FF00D839FF00D749FF00DD3
:10657000659FF00D9927729FB00DE11DF91F639F74
:10658000B00DE11DF91FBD01CF0111240895A1E255
:106590001A2EAA1BBB1BFD010DC0AA1FBB1FEE1F9D
:1065A000FF1FA217B307E407F50720F0A21BB30BE8
:1065B000E40BF50B661F771F881F991F1A9469F764
:1065C00060957095809590959B01AC01BD01CF01C0
:0265D00008952C
:1065D20050000800C0A80001FFFFFF00C0A800088B
:1065E20002CCC0AC00006B139313AA136D146E148B
:1065F200474554002F002F6F6E002F6F6666002FE5
:10660200696D6731002F696D6730006F6666000D36
:106612000D000A0A000D0A0A000A0D0A002403509E
:1066220000000000D4025000000000B404A00000EA
:106632000000740340010000001F5F1D9C1DBC1D73
:106642003A1E691EFF426974416D45746800436CCD
:1066520069656E7420200053746174757320200084
:10666200682C692C6A2C6D2C6E2C008001000000B5
:0666720000007707200084
:00000001FF
